:020000040000FA
:0400000072303A28F8
:040004000034003490
:08000800A000030EA100831209
:100010008B1C32288B1032181428B21C3228643002
:10002000010203183128182800001628172818285C
:1000300019281A281B281C281D281E281F283210A2
:10004000B214A810031005190314AA0DA90DA80DC8
:10005000B10B322832152A08AF002908AE00280853
:10006000AD00B21081010B11210E8300A00E200EF5
:02007000090085
:0C007400203084008001840A6030040207
:10008000031C3C281230B10053218316FF2390003B
:10009000831283160C308505870183128501870141
:1000A000073099000030831691009F008312C830FA
:1000B00083168100831231309000003083168C004B
:1000C000831210308B00842181018E018F010B116E
:1000D0008B100B108C018B177C203219922037214A
:1000E000B40B7A28031085190314BA0DF0303A02C4
:1000F0000319E32085216C286400321808000B1DC9
:1001000008000B11B21032141230B100051D8D28F9
:10011000331483160113831208003310831601175A
:100120008312080032110130B7008B1320303707DB
:1001300083169B001C141A088312A400A500C0306B
:10014000A5061030370783169B001C141A0883126B
:10015000A3000030370783169B001C141A08831273
:10016000A2008B17331CBA2822090339A200A30965
:10017000A409A50922082D02031DDD2823082E024B
:10018000031DDD2824082F02031DCF28013037026C
:10019000031DCF283E18CF283E143F146B2125089D
:1001A0002F02031DDD2801303702031DDC283E1C11
:1001B000DC283E103F146E21DD28B70A02303702DA
:1001C0000318080095280130B600B400B500B70048
:1001D00085018701B2137A217C20B40B002903101A
:1001E00085190314BA0DF0303A0203192729B51FF7
:1001F0008501B51F8701B50B00299630B500322166
:10020000321DEC283211331C0A292D090339AD00A7
:10021000AE09AF092F1CB2132F1CEC28B21BEC281F
:100220002E18EC28B2178B1320303707BC002F088C
:10023000BB00402110303707BC002E08BB00402116
:1002400000303707BC002D08BB0040218B1785010B
:1002500087018121B70AB60102303702031CEC285E
:1002600084210800013037020319712108003F1C66
:1002700008003F101030BC003E08BB0040210800C1
:100280008B133B0883161C159A003C089B005530C5
:100290009D00AA309D009C1464009C184C291C11E0
:1002A00083128B170800831610309B001C141A0849
:1002B0008312BE00FF30D4000230D5000C30D600CF
:1002C000BA30D7003730D800DA30D9006F30DA00D2
:1002D000B830DB0008000130BE000800850187014E
:1002E0000800380933398500B80039093F398700DB
:1002F000B900080011308500B80013308700B9003C
:100300000800B801B9010800080001303E050319D2
:1003100008005C180516DC1885165C190514DC1934
:1003200085145C1A8714DC1A07155C1B0714DC1B88
:1003300087165D180716DD188715E6300E02031CB8
:10034000AB2905168516051485148714071507149F
:100350008716071687158F08031908008F01850176
:1003600087015408DE003822D4005508DE00382208
:10037000D5005608DE00541C3822D6005708DE008F
:10038000D41C3822D7005808DE00541D3822D8006B
:100390005908DE00D41D3822D9005A08DE00541E48
:1003A0003822DA005B08DE00D41E3822DB00CA0BDC
:1003B000E1295408CA00D4185C14D41E5C10D41D62
:1003C0005C10CB0BEB295508CB00D51ADC14551D5E
:1003D000DC10551FDC10CC0BF5295608CC00561A42
:1003E0005C15561F5C11D61D5C11CD0BFF295708FB
:1003F000CD00571ADC15D71FDC11D71DDC11CE0B31
:10040000092A5808CE00D81B5C16D81F5C12D81CCD
:100410005C12CF0B132A5908CF00591ADC16591E4B
:10042000DC12D91FDC12D00B1D2A5A08D000DA19B1
:100430005C17DA1D5C135A1E5C13D10B272A5B086C
:10044000D1005B1ADC175B1EDC13DB1FDC13D20B45
:100450002F2A5608D200D51B5D14D71F5D10D30B71
:10046000372A5708D300D61BDD14D81FDD1008002B
:10047000C001DE080319DE035E184014DE1A4014C2
:100480004008C0015E1C4014DE1E4014C005C00CB4
:040490005E0C0800F6
:084000000F0003000600090097
:02400E00CC01E3
:10420000010003000300030003000200020002009B
:1042100002000000000000000000FF00FF00FF009F
:10422000000000000000000000000000000000008E
:104230000000C000C000C000C000FF00FF00FF0081
:104240000100C300F300CF00FF00C300F300CF0064
:10425000FF00C300F300CF00FF00FF00FF00FF00DE
:10426000FF00FF00FF00FF00FF00FF00FF00FF0056
:10427000FF00FF00FF00FF00FF00FF00FF00FF0046
:10428000FF00FF00FF00FF00FF00FF00FF00FF0036
:10429000FF00FF00FF00FF00FF00FF00FF00FF0026
:1042A000FF00FF00FF00FF00FF00FF00FF00FF0016
:1042B000FF00FF00FF00FF00FF00FF00FF00FF0006
:1042C000FF00FF00FF00FF00FF00FF00FF00FF00F6
:1042D000FF00FF00FF00FF00FF00FF00FF00FF00E6
:1042E000FF00FF00FF00FF00FF00FF00FF00FF00D6
:1042F000FF00FF00FF00FF00FF00FF00FF00AA001B
:00000001FF
